:03000000024F8527
:0C4F850078FFE4F6D8FD758176024FCC71
:101A1B000A53746172743A20004950436F6E6E65BD
:101A2B0063745245510A004950436F6E6E6563747F
:101A3B00003E432C562C43432CC0E4E0EFF2E5F080
:101A4B0020D1E8EDEAEEEC49500A003E432C4D4123
:101A5B00432C25303262583A25303262583A2530C1
:101A6B003262583A25303262583A25303262583A4F
:101A7B0025303262582C4D414320E0E4F0E5F10A69
:101A8B00003E432C5645522C20332E3120EEF220B3
:101A9B0025732025732CC2E5F0F1E8FF2049502077
:101AAB00ECEEE4F3EBFF0A00417072203039203288
:101ABB003030380031323A33343A3535003E432C2E
:101ACB004C442C50524F473A2020202020202020DD
:101ADB0020202020202020202020202020202020FB
:101AEB0020202020202020202020202020202020EB
:101AFB0020202020202020202020202020202020DB
:101B0B00202020202020202020202020202CC4E05A
:101B1B00F2E020EFF0EEF8E8E2EAE828F4E0E9EB97
:101B2B00290A003E2A2C312CCEF1EDEEE2EDFBE53D
:101B3B0020EFE0F0E0ECE5F2F0FB20F1E5F2E5E27E
:101B4B00EEE3EE20E8EDF2E5F0F4E5E9F1E00A0072
:101B5B003E412C4130312C2562752E2562752E2588
:101B6B0062752E2562752C495020E0E4F0E5F120DA
:101B7B00E0E4E0EFF2E5F0E00A003E412C413032C8
:101B8B002C2562752E2562752E2562752E256275A4
:101B9B002C495020E0E4F0E5F120EEF1ED2E20F1A0
:101BAB00E5F0E2E5F0E00A003E412C4130332C2514
:101BBB0062752E2562752E2562752E2562752C4950
:101BCB005020E0E4F0E5F120F0E5E72E20F1E5F020
:101BDB00E2E5F0E00A003E412C4130342C256275E1
:101BEB002E2562752E2562752E2562752CCCE0F1A3
:101BFB00EAE020F1E5F2E80A003E412C4130352CB9
:101C0B002562752E2562752E2562752E2562752C23
:101C1B00D8EBFEE70A003E532C4130362C2562757B
:101C2B002CC2F0E5ECFF20EEE6E8E42E20EAE2E839
:101C3B00F2E0EDF6E8E820282A3130ECF1290A0031
:101C4B003E2A2C312CC4EEEF2E20EFE0F0E0ECE539
:101C5B00F2F0FB20F1E5F2E5E2EEE3EE20E8EDF247
:101C6B00E5F0F4E5E9F1E00A003E422C5330312C6B
:101C7B002562752CC6E4E0F2FC20E7E0EFF0EEF114
:101C8B00E020F1EEE5E4E8EDE5EDE8FF20EEF220F3
:101C9B00F1E5F0E2E5F0E00A003E422C5330322C45
:101CAB002562752CCEE1ECE5ED20F120F1E5F0E2BB
:101CBB00E5F0EEEC20E1E5E720EAE2E8F2E0EDF614
:101CCB00E8E90A003E422C5330332C2562752CCFA9
:101CDB00E5F0E5E7E0EFF3F1EA20EFF0E820EFEED7
:101CEB00F2E5F0E520F1E2FFE7E820F120F1E5F085
:101CFB00E2E5F0EEEC0A003E422C5330342C256228
:101D0B00752CCDE5F220EFE5F0E5E4E0F7E820E413
:101D1B00E8E0E3EDEEF1F2E8EAE820E220F1E5F0AD
:101D2B00E2E5F00A003E422C5330352C2562752C2F
:101D3B00CAE0EDE0EB20F8E8F0EEEAEEE2E5F8E0E1
:101D4B00F2E5EBFCEDEEE3EE20EEE1ECE5EDE00A87
:101D5B00003E532C5330362C25303262582530320E
:101D6B006258253032625825303262582530326243
:101D7B005825303262582C4D414320E0E4F0E5F118
:101D8B0020F8E8F0EEEAEEE2E5F8E0F2E5EBFCED48
:101D9B00EEE3EE20EEE1ECE5EDE00A003E454E44CD
:101DAB000A0044756D7058202020202030302030E0
:101DBB003120303220303320303420303520303653
:101DCB00203037203038203039203041203042202D
:101DDB0030432030442030452030460A003A003A48
:101DEB0020000A0044756D704420202020203030E4
:101DFB002030312030322030332030342030352029
:101E0B0030362030372030382030392030412030E8
:101E1B00422030432030442030452030460A0045D4
:101E2B007272206B657900526420656570726F6DFC
:101E3B000A005264204D454D0A00526420436F64E2
:101E4B00650A0044656275674950204F4E0A00448D
:101E5B00656275674950204F46460A0044656275B6
:101E6B006755736572204F6E0A004465627567553E
:101E7B00736572204F46460A0044656275674D7361
:101E8B0067204F6E0A0044656275674D7367204F7C
:101E9B0046460A00436F6E666967206C6F636B2161
:101EAB000A00577220656570726F6D0A00205361CE
:101EBB00766520656570726F6D210A004572722020
:101ECB004D414321004C6F61643E3E002A003C4172
:101EDB0030313D003C4130323D003C4130333D0020
:101EEB003C4130343D003C4130353D003C413036C7
:101EFB003D003C21003C5330313D003C5330323DE2
:101F0B00003C5330333D003C5330343D003C5330A8
:091F1B00353D003C5330363D0019
:0659A60001730001710015
:10596500C2AFC28E438910758BFF758DB7D2ABD28E
:045975008ED2AF22FD
:03001B00024E5B37
:104E5B00C0E0C083C082C0D0C2AFC28E758BFF755D
:104E6B008DB7201A0675A61E75A6E10571D216E53B
:104E7B007360020573E572D39401400215720576D7
:104E8B00E576540F7050D222E576543F701AD21447
:104E9B00906F48E0601204F0E0D394B4400A908025
:104EAB00007480F0C2AF80FE906F43E0600204F0AC
:104EBB009069BFE0600214F0906F49E0D394014019
:104ECB0003E014F03019020574E575D394644004C3
:104EDB00D21A80020575E570D3940140021570D289
:0C4EEB008ED2AFD0D0D082D083D0E03285
:1008A400C291C290D2B5C21F7D027C007F0712584C
:1008B400F98F27E527646060097D017F601258B1D4
:1008C400D21FE4FDFC7F0B1258F98F27E52730E691
:1008D400097D04E4FF1258D5D21F7D017C007F07F7
:1008E4001258F98F27E5277008FD7FFF1258B1D2FF
:1008F4001F301F03126000C2AFC288C2A8C2AA750B
:10090400890012521A906BFCE0B4FA09A3E064CE99
:1009140070030209A4E4F52774F42527F582E4346E
:100924006BF583E4F00527E527B443EC906BFC7486
:10093400FAF0A374CEF0A374CCF0906C02740AF0B5
:10094400E4A3F0A304F0A3F0906C077403F0A37481
:10095400CCF0906BF874FFF0A3F0A3F0E4A3F09054
:100964006C137405F0E4F527E5272401FFE433FE56
:1009740074F42527F582E4346BF583E0FD12594CB9
:100984000527E527C3944340DFE4F5A775A61E7544
:10099400A6E1907FF0F0A3F09080007480F080FED8
:1009A400D2AF906C077403F0A374CCF0E4906C069F
:1009B400F0124B7BC2B512352CC21A1255D6906C6C
:1009C40013E0C3940350037403F0D21FC221C22066
:1009D400D293201F077E1A7F1B1246AAE4906E331F
:1009E400F0125965C2AFA37408F0906B727424F0CE
:1009F400E4A3F0906BFCE0906B74F0906BFDE090DE
:100A04006B75F0906BFEE0906B76F0906BFFE0906E
:100A14006B77F0906C00E0906B78F0906C01E09054
:100A24006B79F0757201E4906E35F0C21BC21CC282
:100A34001DC21ED2AF75A70775A61E75A6E1125872
:100A44008A201F19AF277E007D031247ABE4FF12F3
:100A54004D117E6C7F33E4FB7D011248A5906F48F5
:100A6400E060037401F0E49069BFF0A37455F0A34F
:100A74007481F0E4F574E4F5759069BFE0700312D5
:100A84003025906F49E0B401119080007410F0E4B7
:100A9400906F49F0D21FC220C221908008E0F52750
:100AA40030E405D21B7410F0E52730E508D21D9020
:100AB40080087420F0E52730E608D21C9080087482
:100AC40040F0E574D394034023908002E4F09080D6
:100AD40001F0908000F0E574D39406400FE4F574BF
:100AE400C217906E35F07572011255D69080A0E051
:100AF40070031252989080B8E070031253129080E1
:100B0400D0E070031253F1908000E07013301B109A
:100B14001245A6906BEFEFF0D39400400312002629
:100B2400908002E07006908000E06005D219020A0D
:100B34007AC219E4F5749069BFE06003020A7A305E
:100B44001D12123F82906BEFEFF0D394004005E04A
:100B5400FF125979201C03020CD9123E0D906BEF41
:100B6400EFF07003020A7A906C33E054BF247F7074
:100B740003020C3C147003020C1424026003020CE4
:100B84006F201F077E1A7F241246AA30237920176C
:100B940076906C0BE07006906C0FE0605B906F3F9A
:100BA400E0FF906C0BE0B50724906F40E0FE906C82
:100BB4000CE0B50618906F41E0FE906C0DE0B506B0
:100BC4000C906F42E0FE906C0EE06E602B906C0F08
:100BD400E06F7033906F40E0FF906C10E0B5072732
:100BE400906F41E0FF906C11E0B5071B906F42E0FD
:100BF400FF906C12E0B5070F906E357401F012008F
:100C040021757201020CD9906F3F74FFF0020CD968
:100C1400906F48E060037401F0906F37E0FF906CD0
:100C240035E06F6003020CD9906F37E004F0E4F50F
:100C340072906E33F0020CD9301703020CD9906C09
:100C440002E07003020A7A1259ADD217E4F57290E9
:100C54006E33F0906F4304F0E4906F36F0A3F0200D
:100C64001F737E1A7F321246AA806A906F48E06032
:100C7400037401F0301752906C33E020E74B906C12
:100C840035E0FF906F36E0FE6F600D906F3EE070D0
:100C940007EE146F703F8013906F36E004F0906B92
:100CA400EFE0FFD3940440031256BD9068BB7482F6
:100CB400F0A37401F0906C35E09068BDF07E687F1D
:100CC400BB7D0312519A020A7A3023092017069039
:100CD4006F3F74FFF0201703020DB5E572706B12BD
:100CE40057A7EF60207E6D7F33906D34E02404FDC0
:100CF40012519A906F3EE06003020A7A906C13E0FE
:100D0400F572020A7A906F43E0D3943C403C906FB2
:100D14003EE07036906F4304F0906B71E0702B12DC
:100D24005993E4906D33F0A37412F0906F37E09010
:100D34006D35F0A374FDF09069C263A201906D3724
:100D440063A2017F121237F9809B1259888F27E51D
:100D540027B401159068BB7483F0E4A3F07E687F28
:100D6400BB7D0212519A020A7AE527D39401401CF2
:100D74009068BB7483F0A37401F0E52724FEA3F00C
:100D84007E687FBB7D0312519A020A7AE572640180
:100D94006003020A7A906E33E004F0E0C3940550D5
:100DA40003020CE9C217E4906E35F0120021020A26
:100DB4007AE57264016003020A7A906E35E0146089
:100DC4004624FE6042147003020EA324046003024E
:100DD4000A7AE4F574202313906E357404F0906E4F
:100DE40033E05401F0757201020A7A9080027410A3
:100DF400F0E4906E35F0906E3304F07572C8906F25
:100E04003F74FFF0020A7A906F3FE07003020E9283
:100E1400906D337480F0906D357401F0E4A3F0A309
:100E240004F0A37430F0A3747BF0E4F527743A253E
:100E340027F582E4346DF583747DF0743B2527F542
:100E440082E4346DF583E4F0E5272407906D34F0F3
:100E54007C6F7D3F906C07E0FAA3E0FB7F021250A9
:100E6400967E6D7F33E5272409FD12519A906F3EDB
:100E7400E0601B1259ADD217E4F572906E33F09016
:100E84006F4304F0E4906F36F0A3F0020A7A906E98
:100E9400357404F0906C13E02432F572020A7A90EF
:100EA40080027410F0757203906E33E06401FFF0F9
:100EB400906E357401F0EF7019906C0FE06013FCC4
:100EC400A3E0FDA3E0FEA3E0FF906F3F1228C6025B
:100ED4000A7A906C0BE0FCA3E0FDA3E0FEA3E0FF24
:0B0EE400906F3F1228C6020A7A80FEC1
:010EEF0022E0
:10002600906C34E0B444047F0180027F00906C330E
:10003600E0B447047E0180027E00EE5F604A906B6A
:10004600FCE0906C35F0906BFDE0906C36F0906BB8
:10005600FEE0906C37F0906BFFE0906C38F0906C9F
:1000660000E0906C39F0906C01E0906C3AF0906C86
:10007600347452F0906B6B63A2019080A863A20166
:100086007F061237F902089A906BEFE0C394085086
:10009600030208A3906BFCE0FF906C35E06F6003F1
:1000A6000208A3906BFDE0FF906C36E06F600302E0
:1000B60008A3906BFEE0FF906C37E06F60030208C8
:1000C600A3906BFFE0FF906C38E06F60030208A31B
:1000D600906C00E0FF906C39E06F60030208A3901B
:1000E6006C01E0FF906C3AE06F60030208A3906C2D
:1000F60034E0B44415906B6BE0B4FF0E63A201903C
:1001060080A863A2017F061237F9906F48E060036A
:100116007401F0906F497464F0906C347452F090EE
:100126006C33E0646D60030202A37BFF7A1A793CAC
:100136001224427BFF7A1A7956906BFCE0F530A3C5
:10014600E0F531A3E0F532A3E0F533A3E0F534A3FF
:10015600E0F5351224427530FF75311A7532B375E4
:1001660033FF75341A7535BF7BFF7A1A798C1224E2
:10017600427BFF7A1A79C81224427BFF7A1B792EBA
:100186001224427BFF7A1B795B906C02E0F530A368
:10019600E0F531A3E0F532A3E0F5331224427BFF0C
:1001A6007A1B7985906C0BE0F530A3E0F531A3E07E
:1001B600F532A3E0F5331224427BFF7A1B79B39024
:1001C6006C0FE0F530A3E0F531A3E0F532A3E0F5DE
:1001D600331224427BFF7A1B79E1906BF8E0F5300D
:1001E600A3E0F531A3E0F532A3E0F5331224427B18
:1001F600FF7A1C7904906BF4E0F530A3E0F531A3A7
:10020600E0F532A3E0F5331224427BFF7A1C792114
:10021600906C13E0F5301224427BFF7A1C794B1266
:1002260024427BFF7A1C7974A223E433F53012242E
:10023600427BFF7A1C79A4906F3EE0F5301224428F
:100246007BFF7A1C79CF906F48E0F5301224427B11
:10025600FF7A1D7902906B71E0F5301224427BFF24
:100266007A1D7930A215E433F5301224427BFF7AE9
:100276001D795C906F38E0F530A3E0F531A3E0F529
:1002860032A3E0F533A3E0F534A3E0F535122442BA
:10029600123C7F7BFF7A1D79A712244222906C3391
:1002A600E0644C70757E1D7FAD1246AA906C3BE0F3
:1002B600F528A3E0F529E4F52B7E1D7FE81246AA72
:1002C6007D03AF29AE281247AB7E1D7FEA1246AAF0
:1002D600E4F52A852982852883E0FF743D252AF5E1
:1002E60082E4346CF583EFF00529E52970020528D0
:1002F600052AE52AB410DC7E6C7F3DE4FB7D1012F6
:1003060048A57E1D7FED1246AA052BE52BC394104A
:1003160040A77E1D7FED1246AA22906C33E0646CE6
:10032600705CF52C7E1D7FEF1246AAE4F52BAF2CF0
:100336007E007D031247AB7E1D7FEA1246AAE4F5D6
:100346002AA82CE6FF743D252AF582E4346CF58351
:10035600EFF0052C052AE52AB410E67E6C7F3DE415
:10036600FB7D101248A57E1D7FED1246AA052BE5E2
:100376002BC3940840B87E1D7FED1246AA22906CCE
:1003860033E0644B7061F52A7425252AF582E4343E
:100396006CF583E060327425252AF582E4346CF529
:1003A60083E0F460237425252AF582E4346CF58312
:1003B600E0FF743B252AF582E4346CF583E0B5074B
:1003C60010052AE52AB408C09069BF7432F0020805
:1003D6009A906C337421F0301F0302089A7E1E7FB8
:1003E6002A1246AA02089A906C33E0B4521A201FC9
:1003F600077E1E7F321246AA906C337472F07E6CB2
:100406007F337D0812511A22906C33E0644970459F
:10041600201F077E1E7F3D1246AA906C3BE0F52802
:10042600A3E0F529E4F52A852982852883E0FF746F
:100436003D252AF582E4346CF583EFF00529E5299C
:1004460070020528052AE52AB480DC7E6C7F337DA0
:100456008A12511A22906C33E064437079A3E064E7
:10046600527046201F077E1E7F451246AA906C3B9F
:10047600E0F528A3E0F529E4F52A85298285288375
:10048600E493FF743D252AF582E4346CF583EFF09E
:100496000529E52970020528052AE52AB480DB7EB0
:1004A6006C7F337D8A12511A22906C34E064576057
:1004B600030208A3906C3BE0F528A3E0F529743D00
:1004C600252AF582E4346CAD82FC7B80AF29AE2808
:1004D60012577302089A906C33E064446003020575
:1004E6006D906C3BE0FF6444700302089AEFB431F0
:1004F6000CC21F7E1E7F4E1246AA02089A906C3BC3
:10050600E0B4300CD21F7E1E7F5A1246AA02089A09
:10051600906C3BE0B4320CD2207E1E7F671246AA56
:1005260002089A906C3BE0B4330CC2207E1E7F75A5
:100536001246AA02089A906C3BE0B4340CD2217E93
:100546001E7F841246AA02089A906C3BE0B4350CD2
:10055600C2217E1E7F911246AA02089A906C3BE049
:10056600FF12001E02089A9069BFE07013201F0751
:100576007E1E7F9F1246AA906C337421F002089A61
:100586009069BF7432F0906C33E0FFB4510A9080EA
:10059600007480F0C2AF80FEEF64577045201F07DD
:1005A6007E1E7FAD1246AA906C3CE0906BEFF0E4A5
:1005B600F52A906BEFE0FFE52AC39F400302089AF5
:1005C600743D252AF582E4346CF583E0FF906C3B9C
:1005D600E0252A246AF582E4346AF583EFF0052AD9
:1005E60080D0906C33E06453600302069C201F07A2
:1005F6007E1E7FB81246AA906BFCE0FF906A73E0FD
:100606006F703C906BFDE0FF906A74E06F70309005
:100616006BFEE0FF906A75E0B50724906BFFE0FF84
:10062600906A76E0B50718906C00E0FF906A77E074
:10063600B5070C906C01E0FF906A78E06F60169049
:100646006C337421F0301F0302089A7E1E7FC71296
:1006560046AA02089AE4F52AE4F575AF2AFE746AFA
:10066600252AF582E4346AF583E0FD12594C052A01
:10067600E52AC394FE40E19080007480F0C2AFE4A6
:10068600907FF0F0A3F0907FFD74AAF0A374FFF0C2
:10069600A37455F080FE906C33E0644F704C906C00
:1006A6003BE0F528A3E0F529E5294528700A201F37
:1006B600077E1E7FD01246AA201F077E1E7FD712F6
:1006C60046AAE4F52A743D252AF582E4346CF583BE
:1006D600E0852982852883F00529E5297002052809
:1006E600052AE52AB480DE02089A906C33E0FFB44E
:1006F60045279080007480F0906C3BE0FDA3E0906D
:100706007FF0CDF0A3EDF0C2AF907FFD74AAF0A309
:1007160074FFF0A37455F080FEEF64656003020871
:100726009A906C3BE0FFA3E0907FF0CFF0A3EFF050
:10073600E4F528F529D3907FF1E09529907FF0E044
:1007460095284020E4F5752529FFE5283401FE8526
:100756002982852883E0FD12594C0529E529700276
:10076600052880D17E1E7FD9125011EF4E602012CF
:100776000003906C02EFF0120003906C03EFF0128E
:100786000003906C04EFF0120003906C05EFF07E0E
:100796001E7FDF125011EF4E6020120003906C0B8B
:1007A600EFF0120003906C0CEFF0120003906C0D4A
:1007B600EFF0120003906C0EEFF07E1E7FE51250F4
:1007C60011EF4E6020120003906C0FEFF012000341
:1007D600906C10EFF0120003906C11EFF012000312
:1007E600906C12EFF07E1E7FEB125011EF4E6020E0
:1007F600120003906BF8EFF0120003906BF9EFF024
:10080600120003906BFAEFF0120003906BFBEFF00F
:100816007E1E7FF1125011EF4E6020120003906B86
:10082600F4EFF0120003906BF5EFF0120003906BFB
:10083600F6EFF0120003906BF7EFF07E1E7FF712D3
:100846005011EF4E6008125579906C13EFF0E4F5F5
:100856002AE4F575E52A2401FFE433FE74F4252A1B
:10086600F582E4346BF583E0FD12594C052AE52A3E
:10087600C3944340DC9080007480F0C2AFE4907F64
:10088600F0F0A3F0907FFD74AAF0A374FFF0A374B8
:0D08960055F080FE7E6C7F337D0812511AF4
:0108A3002232
:10573B00AE07EEC39430400BEED394395005EE24F4
:10574B00D0FF22EEC39461400BEED394665005EE6E
:10575B0024A9FF22EEC39441400BEED3944650058F
:08576B00EE24C9FF22AF062263
:10593200906B6AE004F07006906B69E004F0906B83
:0A59420069E0FEA3E0FF12591622EF
:1000030012593212573BEFC454F0FEC00612593254
:0800130012573BD0E02FFF2241
:10557900E490718AF012593290718BEFF0C3943034
:105589004018E0FFD39439501190718AE024C2F594
:1055990082E43469F583EFF0801190718AE024C2C6
:1055A900F582E43469F583E4F0800C90718AE004B3
:1055B900F0E0D3940840BE753000753100753200B3
:0C55C900E4F5337B017A6979C2123ADB09
:0155D50022B3
:045011008E2D8F2E23
:10501500906B69E4F0A374FFF0125932EF606EF4FF
:10502500606B852E82852D83E493B507EC752F0182
:10503500E52E252FF582E4352DF583E49360259043
:105045006B6AE0252FFF906B69E03400FE1259165C
:10505500E52E252FF582E4352DF583E493B5070478
:10506500052F80CCE52E252FF582E4352DF583E43B
:105075009370A6E52F24FFFFE434FFFE906B6AE0F2
:105085002FF0906B69E03EF07E007F0122E4FEFF89
:0150950022F8
:104B7B007E1E7FFD125011EF4E70037F01227E1FB0
:104B8B007F00125011EF4E600C125932EF24D024DB
:104B9B00FF92238002D2237E1F7F06125011EF4E0D
:104BAB00600C125932EF24D0906F3EF08005E490E8
:104BBB006F3EF07E1F7F0C125011EF4E600C12599E
:104BCB0032EF24D0906F48F08005E4906F48F07E70
:104BDB001F7F12125011EF4E600C125932EF24D07E
:104BEB00906B71F08005E4906B71F07E1F7F181253
:104BFB005011EF4E600C125932EF24D024FF921556
:104C0B008002C215906BFC63A201906F3863A20106
:104C1B007F061237F930153B7E1F7F1E125011EFA6
:104C2B004E6030120003906F38EFF0120003906F5C
:104C3B0039EFF0120003906F3AEFF0120003906F10
:104C4B003BEFF0120003906F3CEFF0120003906FFC
:064C5B003DEFF07F002296
:10562F00906E34E0C3947C503D906E34E0FE04F0F5
:10563F0074722EF582E4346BF583EFF0BF0A279076
:10564F006E34E0FF04F074722FF582E4346BF5834F
:10565F00E4F0906E34E0FF124DBB906E347408F09E
:07566F00906B73E004F022D0
:1055D6009080007480F0906BF463A201F583F582ED
:1055E60063A2017F081237F9906BFC63A2019080D9
:1055F6008863A2017F0A1237F9908092E4F0A374BF
:1056060032F0A37401F0906C06E0FF9080B1F09048
:1056160080E1EFF09080957455F0A3F090800074CF
:0956260001F090800974F0F022FB
:10529800908009E04410F09080A0E0706C9080A1AC
:1052A8007482F09080A874FFF0A3F0A3F0A3F07FBD
:1052B800039080AEEFF07FCBA3EFF07F039080AC3C
:1052C800EFF0A374CBF09080007402F090717C1220
:1052D80028D20000000090717CE0908040F090712E
:1052E8007DE0908041F090717EE0908042F0907176
:1052F8007FE0908043F0A3E4F0A3F0A3F0A3F09044
:095308008018F0A3F0A3F0A3F05B
:015311002279
:1053F100908009E04440F09080D17482F0906C0775
:10540100E0FF9080DEF0906C08E0FF9080DFF0908C
:1054110080027402F09071801228D2000000009086
:105421007180E0908058F0907181E0908059F09007
:105431007182E090805AF0907183E090805BF0A3DC
:10544100E4F0A3F0A3F0A3F0908030F0A3F0A3F078
:02545100A3F0C6
:015453002236
:10531200908009E04420F09080B8E0706C9080B9F1
:105322007482F07F039080C6EFF07FCDA3EFF07F11
:10533200039080C4EFF0A374CDF09080C074FFF0AE
:10534200A3F0A3F0A3F09080017402F09071841294
:1053520028D200000000907184E090804CF090719F
:1053620085E090804DF0907186E090804EF09071D3
:1053720087E090804FF0A3E4F0A3F0A3F0A3F090B5
:095382008024F0A3F0A3F0A3F0D5
:01538B0022FF
:105096008C288D29A907EAFDE975F018A424ACFF30
:1050A600E5F034808F82F583EDF0EBFDE975F018BD
:1050B600A4FFAEF024ACFBEE34808B82F583A3ED27
:1050C600F08529828C83E0FDEF24A8FFEE3480FE74
:1050D6008F82F583EDF08529828C83A3E08F828E03
:1050E60083A3F0852982852883A3A3E0FDE975F0D3
:1050F60018A424A8FFE5F03480FE8F82F583A3A3CD
:10510600EDF08529828C83A3A3A3E08F828E83A3EF
:04511600A3A3F0223D
:06511A008D2DAB07AA0673
:10512000908000E020E57290717CE0FCA3E0FDA39C
:10513000E0FEA3E0F5318E308D2F8C2EAE02AF0352
:105140008E838F8263A201E530540744C0F58385C6
:10515000318263A201AF2D12386BE4FCFDFEE53114
:10516000252DF531EE3530F530ED352FF52FEC35B9
:105170002EF52E908040E52EF0A3E52FF0A3E5302C
:10518000F0A3E531F09080007420F0AF31AE30AD87
:095190002FAC2E90717C1228C690
:0151990022F3
:06519A008D28AB07AA06F8
:1051A000908002E020E572907180E0FCA3E0FDA316
:1051B000E0FEA3E0F52C8E2B8D2A8C29AE02AF03E6
:1051C0008E838F8263A201E52B540744D0F583853B
:1051D0002C8263A201AF2812386BE4FCFDFEE52CA3
:1051E0002528F52CEE352BF52BED352AF52AEC3557
:1051F00029F529908058E529F0A3E52AF0A3E52BAD
:10520000F0A3E52CF09080027420F0AF2CAE2BAD13
:095210002AAC299071801228C615
:015219002272
:024D11008F29E8
:104D1300908001E030E5037F0022907184E0FCA3E2
:104D2300E0FDA3E0FEA3E0F52D8E2C8D2B8C2A90C5
:104D33006F3863A201E52C540744C8F583852D829F
:104D430063A2017F06123881E52D2406F52DE43593
:104D53002CF52CE4352BF52BE4352AF52A906E3609
:104D630063A201E52C540744C8F583852D8263A211
:104D730001AF29123881E4FCFDFEE52D2529F52D2F
:104D8300EE352CF52CED352BF52BEC352AF52A9049
:104D9300804CE52AF0A3E52BF0A3E52CF0A3E52D49
:104DA300F09080017420F0AF2DAE2CAD2BAC2A9087
:074DB30071841228C6AF292C
:014DBA0022D6
:1045A6009081E0E0F5280528052805280528052836
:1045B60005280528052805280528908010E0F52BF4
:1045C600A3E0F52CA3E0F52DA3E0F52E9081E1E024
:1045D600F52805280528052805280528052805287D
:1045E600052805280528908014E0F52FA3E0F5306E
:1045F600A3E0F531A3E0F532E531B52D08E532B596
:104606002E037F0022E4F528E531540744E0F583C4
:1046160085328263A201906C3363A2017F0812384F
:10462600B1906C3563A201906B6B63A2017F061299
:1046360037F9906C33E0F529A3E0F52AE4F52890E4
:104646006C33E0702AA3E024F8F528E531540744DA
:10465600E0F58385328274082582F582E43583F598
:104666008363A201906C3363A201AF281238B1AE06
:1046760029E4FCFDE532252AF532E5313EF531ED3A
:104686003530F530EC352FF52F908014E52FF0A35B
:10469600E530F0A3E531F0A3E532F09080007440F8
:0346A600F0AF284A
:0146A90022EE
:103E0D009081E6E0F52805280528052805280528D0
:103E1D0005280528052805280528908028E0F52B7C
:103E2D00A3E0F52CA3E0F52DA3E0F52E9081E7E0BE
:103E3D00F52805280528052805280528052805281D
:103E4D0005280528052890802CE0F52FA3E0F530F6
:103E5D00A3E0F531A3E0F532E4F528E531B52D0AFF
:103E6D00E532B52E05C21C023F67E531540744F01B
:103E7D00F58385328263A201906C3363A2017F08C2
:103E8D001238B1906C33E0F529A3E0F52AE52A4507
:103E9D002970099080027410F07F0022906F3FE02E
:103EAD00FFF4602D906C35E06F7076906F40E0FF01
:103EBD00906C36E06F706A906F41E0FF906C37E068
:103ECD006F705E906F42E0FF906C38E06F60228003
:103EDD0050906C35E0906F3FF0906C36E0906F40F5
:103EED00F0906C37E0906F41F0906C38E0906F423D
:103EFD00F0906C33E0702AA3E024F8F528E53154F6
:103F0D000744F0F58385328274082582F582E43505
:103F1D0083F58363A201906C3363A201AF2812383D
:103F2D00B1AE29E4FCFDE532252AF532E5313EF549
:103F3D0031ED3530F530EC352FF52FAF2EAE2DADF3
:103F4D002CAC2BAB32AA31A930A82FD31228954017
:103F5D00099080027410F07F002290802CE52FF0E4
:103F6D00A3E530F0A3E531F0A3E532F090800274C3
:043F7D0040F0AF2839
:013F8100221D
:103F82009081E3E0F528052805280528052805285D
:103F92000528052805280528052890801CE0F52B12
:103FA200A3E0F52CA3E0F52DA3E0F52E9081E4E04B
:103FB200F5280528052805280528052805280528A7
:103FC200052805280528908020E0F52FA3E0F5308C
:103FD200A3E0F531A3E0F532E4F528E531B52D0A89
:103FE200E532B52E05C21D0240CDE531540744E845
:103FF200F58385328263A2019068BF63A2017F0EBE
:104002001238C79068BFE0F529A3E0F52A9068C787
:10401200E0FFF46045906F38E0FEEF6E706EA3E053
:10402200FF9068C8E06F7064906F3AE0FF9068C9D3
:10403200E06F7058906F3BE0FF9068CAE06F704C81
:10404200906F3CE0FF9068CBE06F7040906F3DE076
:10405200FF9068CCE06F60048032D2D99068BFE0F4
:10406200702AA3E024F2F528E531540744E8F583E9
:10407200853282740E2582F582E43583F58363A24C
:10408200019068BF63A201AF281238C7AE29E4FCD1
:10409200FDE532252AF532E5313EF531ED3530F5D3
:1040A20030EC352FF52FAF2EAE2DAD2CAC2BAB3225
:1040B200AA31A930A82FD31228955006E52A4529FE
:1040C20070099080017410F07F0022908020E52F0B
:1040D200F0A3E530F0A3E531F0A3E532F0908001E2
:0540E2007440F0AF285E
:0140E70022B6
:0446AA008E318F328C
:1046AE00E4F533F534908000E030E5110534E5345F
:1046BE0070020533D39488E533941340E89080005C
:1046CE00E030E5030247AA90717CE0FCA3E0FDA375
:1046DE00E0FEA3E0F5388E378D368C35E538FFE5F4
:1046EE00375407FEE42FF534EE34C0F533853482AB
:1046FE00F5837423F00534E534700205335333C764
:10470E00F582853383740AF00534E534700205337F
:10471E005333C7906BFC63A2018533838534826368
:10472E00A2017F0612386B74062534F534E4353356
:10473E00F53385318385328263A2018533838534D7
:10474E008263A20112384FE4FCFDFE90717CE0F80A
:10475E00A3E0F9A3E0FAA3E02FFFEE3AFEED39FD58
:10476E00EC38FCEF2408FFE43EFEE43DFDE43CFCA7
:10477E0090717C1228C690717CE0908040F0907110
:10478E007DE0908041F090717EE0908042F09071DB
:0C479E007FE0908043F09080007420F0D9
:0147AA0022EC
:0648A5008E2E8F2F8D30D6
:1048AB00E4F531F532908000E030E5110532E53268
:1048BB0070020531D39488E531941340E890800061
:1048CB00E030E50302499890717CE0FCA3E0FDA386
:1048DB00E0FEA3E0F5368E358D348C33E536FFE5FF
:1048EB00355407FEE42FF532EE34C0F531853282B4
:1048FB00F5837423F00532E532700205315331C76D
:10490B00F582853183EBF00532E5327002053153C8
:10491B0031C7906BFC63A20185318385328263A220
:10492B00017F0612386B74062532F532E43531F50A
:10493B0031852E83852F8263A20185318385328257
:10494B0063A201AF3012386B74082530F530FFE4E9
:10495B00FCFDFEE5362FF536EE3535F535ED353408
:10496B00F534EC3533F533908040E533F0A3E53483
:10497B00F0A3E535F0A3E536F09080007420F0AF9E
:0D498B0036AE35AD34AC3390717C1228C6C9
:0149980022FC
:024DBB008F4126
:104DBD00E4F542F543908000E030E5110543E5430D
:104DCD0070020542D39488E542941340E890800028
:104DDD00E020E57990717CE0FCA3E0FDA3E0FEA36B
:104DED00E0F5478E468D458C44E547FFE546540773
:104DFD00FEE42FF543EE34C0F542906B7263A201D1
:104E0D0085428385438263A201AF4112386BE4FC76
:104E1D00FDFEE5472541F547EE3546F546ED3545B1
:104E2D00F545EC3544F544908040E544F0A3E54567
:104E3D00F0A3E546F0A3E547F09080007420F0AFB5
:0D4E4D0047AE46AD45AC4490717C1228C6BE
:014E5A002235
:0647AB008E2D8F2EAB05E0
:1047B100E4F52FF530908000E030E5110530E5306B
:1047C1007002052FD39488E52F941340E890800060
:1047D100E030E5030248A490717CE0FCA3E0FDA376
:1047E100E0FEA3E0F5348E338D328C31E534FFE504
:1047F100335407FEE42FF530EE34C0F52F853082B7
:10480100F5837423F00530E5307002052F532FC76F
:10481100F582852F83EBF00530E5307002052F908E
:104821006BFC63A201852F8385308263A2017F0621
:1048310012386B74062530F530E4352FF52F532FE0
:10484100C7E52D853082852F83F00530E530700274
:10485100052F532FC7F582852F83E52EF00530E50F
:10486100307002052F532FC7E534240AF534E4359F
:1048710033F533E43532F532E43531F531908040AA
:10488100E531F0A3E532F0A3E533F0A3E534F09090
:1048910080007420F0AF34AE33AD32AC3190717C16
:0348A1001228C614
:0148A40022F1
:10545400908009E04480F09080E97401F07F099025
:1054640080F6EFF0A37464F09080037402F09080EF
:1054740000E020E1F99070781228D200000000903A
:105484007078E0908064F0907079E0908065F0909E
:10549400707AE0908066F090707BE0908067F0A373
:1054A400E4F0A3F0A3F0A3F090803CF0A3F0A3F009
:0254B400A3F063
:0154B60022D3
:104999009081E9E0F52E052E052E052E052E052E12
:1049A900052E052E052E052E052E908034E0F52FB7
:1049B900A3E0F530A3E0F531A3E0F5329081EAE018
:1049C900F52E052E052E052E052E052E052E052E56
:1049D900052E052E052E908038E0F533A3E0F53439
:1049E900A3E0F535A3E0F536E535B53108E536B58B
:1049F90032037F0022E4F52EE535540744F8F583A8
:104A090085368263A20190707C63A2017F06123809
:104A1900DF90707CE064686014908038E52FF0A323
:104A2900E530F0A3E531F0A3E532F0804C90707DDC
:104A3900E02402F52EE535540744E0F583853682F6
:104A490063A20190707C63A201AF2E1238DFE4FCEF
:104A5900FDFEE536252EF536EE3535F535ED3534E1
:104A6900F534EC3533F533908038E533F0A3E5348C
:104A7900F0A3E535F0A3E536F09080037440F0AF7C
:014A89002EFE
:014A8A002209
:024A8B008F2E6C
:104A8D009080E8E0640660037FFF22907078E0FC80
:104A9D00A3E0FDA3E0FEA3E0F5328E318D308C2F27
:104AAD00E4FFFEFDFCAB32AA31A930A82FC31228BA
:104ABD009570609081F9E0F52F907078E0FCA3E09F
:104ACD00FDA3E0FEA3E0FFE4FAF9F8EF2401FFEA0D
:104ADD003EFEE93DFDE83CFC9070781228C69070D2
:104AED0078E0FCA3E0FDA3E0FEA3E0FFE4F8EF24F3
:104AFD0001FFEA3EFEE93DFDE83CFC90707812288E
:104B0D00C6908064E0F52FA3E0F530A3E0F531A366
:104B1D00E0F53290707C63A201E531540744D8F57D
:104B2D008385328263A201AF2E123899E4FCFDFE1B
:104B3D00E532252EF532EE3531F531ED3530F530E6
:104B4D00EC352FF52F908064E52FF0A3E530F0A321
:104B5D00E531F0A3E532F09080037420F0AF32AE72
:0D4B6D0031AD30AC2F9070781228C67F005B
:014B7A002218
:10591600E5D220E0FBC2AF438E2075D2028F828E85
:0B59260083E0FFE4F5D2538EDFD2AF28
:015931002253
:10594C00E5D220E0FBC2AF43D2028F828E83EDF012
:09595C0075D25063D250D2AF2283
:10521A00E4FDED2401FFE433FE12591674F42DF572
:10522A0082E4346BF583EFF00DBD3FE6E4FDED2437
:10523A007FFFE433FE12591674EA2DF582E43469CD
:10524A00F583EFF074EA2DF582E43469F583E070B2
:10525A001B74EA2DF582E43469F5837420F074EB4B
:10526A002DF582E43469F583E4F080040DBD80BE37
:10527A00E4906A69F0FDEDFF7E00125916746A2DFA
:0D528A00F582E4346AF583EFF00DBDFEE916
:0152970022F4
:025773008B2D7C
:10577500A2AF9224C2AF85A22E53A2FE8E838F8242
:1057850005A28C838D8274091238F5E52D53A2FE8E
:1057950043A2201238F753A2DF852EA2A22492AF8E
:0157A500FF04
:0157A60022E0
:1058F900A2AF9224C2AF8C838D82EF1238F543A2F6
:0C590900201238F753A2DFA22492AFFF57
:01591500226F
:0258B1008F283E
:1058B300A2AF9224C2AFE4F5838D8274061238F549
:1058C300E52843A2201238F753A2DFA22492AF7F28
:0158D30001D3
:0158D40022B1
:0258D5008F281A
:1058D700A2AF9224C2AFE4F5838D82740A1238F521
:1058E700E52843A2201238F753A2DFA22492AF7F04
:0158F70001AF
:0158F800228D
:10371E00A907E7FFA805EF93C3966008403B74FC2A
:10372E002FFF80F00F08EF93C3966008402B74FBB9
:10373E002FFF80E00F08EF93C3966008401B74FACA
:10374E002FFF80D00F08EF93D3966008400B74F9CB
:10375E002FFF80C01F1F1F1F1FEF54FEF80303F71C
:10376E00E893FC08E893FD08E893FE08E893FF222F
:10377E0009E993C39D6008402974FB29F980F1097A
:10378E00E993C39E6008401A74FA29F980E209E9A8
:10379E0093D39F6008400B74F929F980D319191936
:1037AE001919E9C313C313FF22740093F8ECC398DD
:1037BE004024701F740193F8EDC39840197014746F
:0E37CE000293F8EEC398400E7009740393F84E
:1037DC00EFC39840037F00227F0122EDF8E6F0084A
:1037EC00A3DFFA22EDF8E0F608A3DFFA22E0A363E8
:1037FC00A201F0A363A201DFF475A2002263A2016F
:10380C00F0A363A20122E0A363A201F0A363A201CF
:10381C00E0A363A201F0A363A201E463A201F0A3FD
:10382C0063A201DFE175A20022E0A363A2016DFE99
:10383C00936CFDEE058393FC158363A201DFEA759F
:10384C00A200227F00E493A363A201F00F600CA3FB
:10385C00E583C2E3F58363A20180EA75A20022E04E
:10386C00A363A201F0A3E583C2E3F58363A201DFA6
:10387C00EE75A20022E0A363A201F0A3E583C2E4EB
:10388C00D2E3F58363A201DFEC75A20022E0A3630F
:10389C00A201F0A3E58344F8C2E5F58363A201DF3E
:1038AC00EC75A20022E583C2E3F583E0A363A201D9
:1038BC00F0A363A201DFEE75A20022E583C2E4D27D
:0A38CC00E3F583E0A363A201F0A37B
:1038D60063A201DFEC75A20022E58344F8F583E0DC
:1038E600A363A201F0A363A201DFEE75A20022F991
:1038F60022C002C004C00612FFF0D006D004D002D7
:01390600229E
:104EF7000A536572763A004572724C656E210A0054
:104F0700205544502054696D654750530A00200AC4
:104F1700444154414752414D3A20002043414E20DD
:104F270054696D654750530A002054726173735377
:104F3700656E644552520A000ACEF8C4EBE8EDFBF1
:104F470043414E210A000A45727241647243414E41
:104F57003A000A00205265496E69742043414E0A9F
:104F6700002043414E283029203E20544F210A007B
:0E4F770020545520300A0020545520310A00E5
:03001E00E4FF22DA
:10586200C2A9438902758C48758A4875D90475DBCB
:105872004875DC4875DD4875DE48E4F5E9F5F9D28E
:08588200D9C2DAD28CD2DE2279
:10580900C2D9906F5EE07013E5E92419F5EB30D742
:1058190006E5F904F5FB2285F9FB22E5E924C8F53B
:0E582900EB30D706E5F904F5FB2285F9FB22EA
:10567600C2D9906F5EE0702C303116E5E92432F520
:10568600EB30D707E5F904F5FB800385F9FBC2315A
:1056960022E5E92405F5EB30D706E5F904F5FB220A
:1056A60085F9FB22E5E92432F5EB30D706E5F90466
:0756B600F5FB2285F9FB2240
:10588A00125862906F5EE0C39464500612538C12F1
:10589A005809120022D230E4F559907076F0F54892
:0758AA00F55DC231F55B2240
:1056BD00EF24FCF548201F127E4E7FF71246AA7E7E
:1056CD006C7F37E4FBAD481248A5E548D3940D40F7
:1056DD0010201F077E4E7FFE1246AAE4F548D22EFB
:1056ED0022906C3763A20190706663A201AF4812DD
:0556FD0037F9C22E2266
:0F597900D3EF6480948D5006E55D70028F5D2240
:1030250020D903023102203003023102E55D6052EE
:103035009068BF540FFF7D4A1237F0E54A6401706E
:103045001E9068C7E0B4FF0ED232201F127E4F7F5C
:10305500071246AA8009303206E4F55D02310212F4
:1030650058091254B7201F077E4F7F151246AA2014
:103075001F0B7E687FBFE4FBAD5D1248A5E4F55DDF
:10308500807BE548604390706AE02405F528D39479
:103095000D4007E4F548D22E8063907066E528540C
:1030A5000FFF7D4A1237F0E54A30E702D231E54A93
:1030B500B40109303206E54D640160031254B712BC
:1030C5005809E4F548D22E8034E55A601E906F4ABF
:1030D500540FFF7D4A1237F0E54AB401032032034D
:1030E5001254B7125809E4F55A801220010C906F5A
:1030F5005EE0C3946450031255191258091240E852
:103105008F28EF70030231C9125676E4F55BE54A64
:10311500B4010CD232201F077E4F7F221246AAE54A
:103125005CC394C8502D30172AE54AB4420DE54DCD
:10313500B40208906B71E064016018745F255CF55A
:1031450082E4346FF583E528255CF55C7D4AAF287C
:103155001237E7301521E54A20E71C906E367D4A87
:10316500AF281237E7AF28124D11EF700A201F075D
:103175007E4F7F301246AAE54A54817047E528D331
:10318500940D400C201F3D7E4F7F3F1246AA803490
:10319500E54CD394074028201F2A7E4F7F4D1246C9
:1031A500AA9069C27D4AAF281237E77E697FC2E4DB
:1031B500FBAD281248A57E4F7F591246AA8005AF60
:1031C50028122D4930222C90661EE0C394FA500334
:1031D500E004F030141B906F5EE0C3946450120558
:1031E5005BE55B94F0400A9080007480F0C2AF808C
:1031F500FEC2222016030232F0E5596031D3940154
:10320500400415598028907076E004F0E0D39403CB
:10321500400D201F077E4F7F5B1246AA12588A2059
:103225001F077E4F7F681246AAE4F559D230302F2A
:1032350043E55A703F906F4A04F0A37408F0A374F5
:1032450080F0A37401F0A37406F0907061E0906FB4
:103255004FF0907062E0906F50F0907063E0906F67
:1032650051F0907064E0906F52F0E4A3F0A3F07514
:103275005A0BC22F302D7290705FE07035E55A7091
:1032850031906F4A7442F0A37408F0907060E0903A
:103295006F4CF0907065E0906F4DF0A37401F07580
:1032A5005A06201F077E4F7F771246AA90705FE06F
:1032B50004F090705FE06402702FE55A702B906FF8
:1032C5004A7402F0A37408F0907060E0906F4CF0BF
:1032D500A3F0A37401F0755A06201F077E4F7F7E69
:1032E5001246AA90705FE004F0C216121F24C214A1
:0132F50022B6
:1057A700E55C602CE4906D33F0A3E55CF0906F3717
:1057B700E0906D35F0A37419F0906F5F63A20190CC
:1057C7006D3763A201AF5C1237F9E4F55C7F012204
:0357D7007F00222E
:0B598800302E05C22E7F01227F00227E
:0100210022BC
:0659AD00E4F55CF5482260
:0A599300E49069C2F0A3F0A3F02233
:1057DA002043616E457247495400200A004572729F
:1057EA004C656E43616E21000A002043616E45726A
:0F57FA0072434821000A205265714572722100E6
:1040E800E59B541F6020201F1A7E577FDA1246AACC
:1040F800E59B541FFF7E007D031247AB7E577FE48C
:104108001246AAE4F59BE5BA30E010E4F5B375B1C0
:1041180080F5B2D230F559907076F0E5CFF470039F
:1041280002423D752A01E4F529E5CFF4552A7003CA
:1041380002422BE529C454F0F5B1E5B2547F64205E
:1041480060030241FCE5B3540FF54E85BC4AE5BD5A
:10415800541FFF131313541FFFE5BD54E044184FB9
:10416800F54BE5BDC43354E0FFE5BE131313541FEC
:104178004FF54CE5BEC43354E0FFE5BF13131354A9
:104188001F4FF54D85A34F85A35085A35185A35295
:1041980085A35385A35485A35585A356E4F5B2207A
:1041A800010CE54A547EB54A0575B350800375B3D2
:1041B800D0E54E700AE54A547EB54A037F002230A6
:1041C8000108E54A30E7037F0022E54ED394084012
:1041D8001D201F177E577FE71246AAAF4E7E007D2F
:1041E800031247AB7E577FF21246AA7F0022E54EA4
:1041F8002405FF22E5B2549F6023201F207E577FAD
:10420800F41246AAAFB27E007D031247ABAFB37E6D
:10421800007D031247AB7E577FF21246AAE4F5B23F
:1042280075B3D0E52A25E0F52A0529E529C39408C0
:0742380050030241317F0039
:01423F00225C
:1054B700906F5EE0C39464505675B180E4F5B3F520
:1054C700B2854ABCE54CC4135407FFE54B54E04F83
:1054D700F5BDE54C33333354F8FFE54DC41354079A
:1054E7004FF5BEE54D33333354F8F5BF854FA385EC
:1054F70050A38551A38552A38553A38554A38555EE
:10550700A38556A3E54E540F2450F5B375590AC227
:02551700302240
:1055190075B190E5B220E613201F107E577FFF1268
:1055290046AAAFB27E007D031247ABE4F5B3F5B2EC
:1055390074902512F582E43461F583E0F5BCE4F555
:10554900BD74912512F582E43461F583E0FF3333AC
:105559003354F8F5BE75BF780512051274902512FB
:10556900F582E43461F583E07002F51275B35022D7
:09599D00EF6003C29622D29622AB
:10538C0043AB01C2E8C2EAE4FFEFC454F0F5B1C389
:10539C00EF64809488500575B3D08003E4F5B3E4D2
:1053AC00F5B2F5BCF5BDF5BEF5BFF5C4F5C5F5C652
:1053BC00F5C7F5A3F5A3F5A3F5A3F5A3F5A3F5A3FD
:1053CC00F5A30FBF0EC3906F5EE0FF25E0F5B4753B
:1053DC00B50C75B66C75A11275AB0275C13E75C373
:0453EC00FF75C20384
:0153F000229A
:1039070000000000000000000000000000000000B0
:103917003FF3630041D5E80043B71B8045984F004C
:1039270047798280495C07804B3D3B004D1E6E8086
:103937004EFFA20050E2270052C35A8054A48E00C3
:103947005685C180586846805A497A005C2AAD80FE
:103957005E0BE1005FEE660061CF998063B0CD003A
:1039670065920080677485806955B9006B36EC8075
:103977006D1820006EFAA50070DBD88000000000EB
:103987000028DE80004DC8800076A700009E340026
:1039970000C7123000EE9F8001177E0001405C8057
:1039A7000167E9800190C80001B8550001E1338043
:1039B700000000000028DE80004F1A000077F88022
:1039C700009F858000C8640000EFF1000118CF80D8
:1039D7000141AE0001693B000192198001B9A6803F
:1039E70001E2850000000000000151800002A300F1
:1039F7000003F48000054600000697800007E900F1
:103A070000093A80000A8C00000BDD80000D2F00B2
:103A1700000E8080000FD200001123800012750075
:103A27000013C68000151800001669800017BB0038
:103A370000190C80001A5E00001BAF80001D0100FA
:103A4700001E5280001FA4000020F58000224700BE
:103A5700002398800024EA0000263B8000278D0081
:103A67000028DE800000000000000E1000001C206F
:103A770000002A3000003840000046500000546023
:103A8700000062700000708000007E9000008CA033
:103A970000009AB00000A8C00000B6D00000C4E043
:103AA7000000D2F00000E1000000EF100000FD2050
:103AB70000010B300001194000012750000135605B
:103AC70000014370000151801F1C1F1E1F1E1F1F76
:043AD7001E1F1E1F71
:10437500E50825E025E02407F582E43439F58312C4
:1043850028A68F118E108D0F8C0EE508540370280A
:10439500E50D25E025E024B3F582E43439F58312F3
:1043A50028A6EF2511F511EE3510F510ED350FF5B1
:1043B5000FEC350EF50E8026E50D25E025E0247F72
:1043C500F582E43439F5831228A6EF2511F511EEAF
:1043D5003510F510ED350FF50FEC350EF50EE50A38
:1043E50025E025E024E7F582E43439F5831228A693
:1043F500EF2511F511EE3510F510ED350FF50FEC34
:10440500350EF50EE50BC3940C402AE51124C0F5D5
:1044150011E51034A8F510E4350FF50FE4350EF568
:104425000EE50B24F4FF7E007C0E7D1012273CAABE
:1044350006AB07800FAF0B7E007C0E7D1012273C6C
:10444500AA06AB07AE02E4FCFDE5112BF511E5105C
:104455003EF510ED350FF50FEC350EF50EE50C7547
:10446500F03CA4FFAEF0E4E5112FF511E5103EF5A3
:1044750010ED350FF50FEC350EF50EE4FEE51125C3
:1044850009F511EE3510F510ED350FF50FEC350E7C
:02449500F50E22
:014497002202
:1042400090718CE0F50825E025E02407F582E43440
:1042500039F583E508D3941F501DAF11AE10AD0F93
:10426000AC0E1237B7EF700F74042582F582E43577
:1042700083F583050880DC74FC2582F58274FF35A4
:1042800083F583AF821228B6C3E5119BF511E510C3
:104290009AF510E50F99F50FE50E98F50E1508E55E
:1042A000081490718CF0E508540370059039B780BC
:1042B00003903983750D307F0D7D0E12371EA804D3
:1042C000A905AA06C3E5119FF511E5109AF510E5B9
:1042D0000F99F50FE50E98F50E050D9039EBAF111E
:1042E000AE10AD0FAC0E7B007A00797C12377E8F5A
:1042F0000AEF25E025E024EBF582E43439F583125A
:1043000028B6C3E5119BF511E5109AF510E50F9954
:10431000F50FE50E98F50E050A903A6BAF11AE1049
:10432000AD0FAC0E7B007A00795C12377E8F0BEFFD
:1043300025E025E0246BF582E4343AF5831228B6B3
:10434000C3E5119BF511E5109AF510E50F99F50FEE
:10435000E50E98F50EAE10AF117C007D3C12274E95
:104360008D09AE10AF117C007D3C12274E8E108F50
:054370001185110C2273
:1014DF003E2A2C312CCFE0F0E0ECE5F2F0FB20F3CC
:1014EF00EFF0E0E2EBFFFEF9E5E3EE20EAEEEDF2DE
:1014FF00F0EEEBEBE5F0E020CACF20C8F1E5F2FC0F
:10150F000A003E4C2C6B30312C25732C43EAEEF045
:10151F00EEF1F2FC20EDE020F8E8EDE52043414E3E
:10152F002C30202D20353030EAE1283530EC292CB5
:10153F0031202D203530EAE128353030EC290A00F2
:10154F0030202D20353030EAE1283530EC290031BC
:10155F00202D203530EAE128353030EC29003E537C
:10156F002C6B30322C2562752CCCE0EAF12E20E06A
:10157F00E4F0E5F120E1EBEEEAE020D2D128302DC6
:10158F0038290A003E532C6B30332C2562752CCC36
:10159F00E0EAF12E20E0E4F0E5F120E1EBEEEAE005
:1015AF0020D2C8D228302D38290A003E532C6B3058
:1015BF00342C2562752CCCE0EAF12E20E0E4F0E526
:1015CF00F120E1EBEEEAE020D2D328302D38290AC2
:1015DF00003E422C6330312C2562752CC2F2EEF0A6
:1015EF00E8F7EDFBE920EAEEEDF2F0EEEBEBE5F0DC
:1015FF0020EDE020F8E8EDE50A003E2A2C312CCF53
:10160F00E0F0E0ECE5F2F0FB20EFF0EEF2EEEAEEC8
:10161F00EBE020CCDDCA203837302D352D3130347A
:10162F0028313031290A003E4C2C6B30352C256C7B
:10163F00752C2831303129D1EAEEF0EEF1F2FC2091
:10164F00EEE1ECE5EDE020EDE020EFEEF0F2F32C33
:10165F003130302C3230302C3330302C3630302C7F
:10166F00313230302C323430302C343830302C3959
:10167F003630302C31393230302C33383430302C46
:10168F0035373630302C3131353230300A003E5359
:10169F002C6B30362C2562752C2831303129CDEE4C
:1016AF00ECE5F020F1F2E0EDF6E8E80A003E532C0D
:1016BF006B30372C2562752CC0E4F0E5F1204153D7
:1016CF0044550A003E532C6B30382C256C752CCDAD
:1016DF00E0F7E0EBFCEDFBE920E0E4F0E5F120D2F0
:1016EF00D10A003E532C6B30392C256C752CCDE074
:1016FF00F7E0EBFCEDFBE920E0E4F0E5F120D2C8E8
:10170F00D20A003E532C6B31302C256C752CCDE05A
:10171F00F7E0EBFCEDFBE920E0E4F0E5F120D2C8C7
:10172F00C80A003E532C6B31312C256C752CCDE043
:10173F00F7E0EBFCEDFBE920E0E4F0E5F120D2D39C
:10174F000A003E422C6B31322C2562752CD0E0E71B
:10175F00ECE5F020C0D1C4D33D322831290A003E38
:10176F00422C6B31332C2562752CD0E0E7ECE5F081
:10177F0020EFF0E8F7E8EDFB20EFE5F0E5E4E0F728
:10178F00E83D322831290A003E422C6B31342C259A
:10179F0062752CD0E0E7ECE5F020E0E4F0E5F1E055
:1017AF0020EEE1FCE5EAF2E03D332832290A003E63
:1017BF00422C6B31362C2562752CCFE5F0E5E4E039
:1017CF00F7E020D2C8D220F120E2F0E5ECE5EDE51C
:1017DF00EC0A003E422C6B31382C2562752C2831D7
:1017EF0030342954435020EAEBE8E5EDF20A003E8D
:1017FF00532C6B31372C2562752C2831303429CA84
:10180F00EEEB20EFE0EAE5F2EEE220EDE020EAE297
:10181F00E8F20A003C21003C6B30313D003C6B305C
:10182F00323D003C6B30333D003C6B30343D003C6F
:10183F006330313D003C6B30353D003C6B30363D05
:10184F00003C6B30373D003C6B30383D003C6B301B
:10185F00393D003C6B31303D003C6B31313D003C3C
:10186F006B31323D003C6B31343D003C6B31333DCD
:10187F00003C6B31353D003C6B31363D003C6B31EC
:10188F00373D003C6B31383D0052657374617274A3
:10189F0020424C0A0043414E205455204F4B0A0022
:1018AF0043414E205455205265710A00496E6974A8
:1018BF005443500A00436F6E6E6563745443500A6D
:1018CF00004C697374656E5443500A00534F434B79
:1018DF005F5443505F45535441424C49534845442C
:1018EF000A002054552054696D654F5554210A0044
:1018FF000A2D3E20000A3E000A3ED1E1F0EEF1CA69
:10190F00E0EDE0EBE0203A3C28CAE2F229000A3E83
:10191F00D1E1F0EEF1CFF0EEF6E5E4F3F0203A3C52
:10192F0028CAE2F229003A3C28CAE2F229000A3E0C
:10193F00D1F2E0F2F3F1CAE0EDE0EBE03F203A3C08
:10194F0028CAE2F229000A3EC7E0EFF0EEF13A00B2
:10195F003C28CDE5F2C4E0EDEDFBF529003E3F3F1D
:10196F003F3A0020D2D3200020C2FBE1EEF020004E
:10197F0020C8F1EFEEEBEDE8F2FC200020CEF2EC08
:10198F00E5EDE0200020C2F0E5ECFF200020CEEFD7
:10199F00F0EEF1200020C7E0E2E5F0F8E5EDE8E534
:1019AF00C8EDE8F6E8E0EBE8E7E0F6E8E82000202D
:1019BF00CAE2E8F2D2D3200020CEF8E8E1EAE0D282
:1019CF00D3200020D2D320C3EEF2EEE2EE2000208F
:1019DF00D2D320C2FBEFEEEBEDE5EDEE200020D2EF
:1019EF00D1F1200020C0EAF2E2F6CEEFF0EEF1E006
:1019FF00200020D2D1F6200020D2C8D2F62000201D
:0C1A0F00D2C8C8200020D2C8D2F12000AC
:03002300024498FC
:0B449800C0E0C083C082C0D075D01807
:1044A300209803024567C298757301AF99300603DC
:1044B30002459DD291200228BF680DD202D20E750B
:1044C3006400756800024567EF6410600302456786
:1044D300D202D20F756F0275680375640002459DA1
:1044E300E56870078F6F056802459DE568B4010FA5
:1044F300E56FB51F05056802459DC20202459DE5AE
:1045030068B4020AEF646860CEC20202459DE568A2
:10451300B4031E74792569F582E43466F583EFF0FC
:1045230005692564F564156FE56F706E7568048021
:1045330069E568B4040DE564B51F040568805BC2D2
:10454300028057E568B4051CBF160ED20685696F55
:10455300756900C202C2918041C20FC20E75690023
:10456300C202803630993330032E90618EE0FFE52E
:104573006BC39F4008C203D210C290801BD29074B9
:10458300B9256BF582E43467F583E0F56E526EA2CC
:0A459300D0929B856E99056BC299CA
:09459D00D0D0D082D083D0E032EE
:103C7F007BFF7A1479DF122442906F5EE070147527
:103C8F0030FF75311575324F7BFF7A15791112247C
:103C9F004280127530FF75311575325E7BFF7A15D4
:103CAF0079111224427BFF7A15796D90618FE0F5BF
:103CBF00301224427BFF7A157993906102E0F53040
:103CCF001224427BFF7A1579BA906101E0F5301228
:103CDF0024427BFF7A1579E0A201E433F5301224F8
:103CEF00427BFF7A1679091224429068B9E0FEA34D
:103CFF00E0FFC3E49FFFE49EFEAB07FA3395E0F9C4
:103D0F00F87F007E8C7D0A7C001227F58F338E3270
:103D1F008D318C307BFF7A1679361224427BFF7AF5
:103D2F0016799D906413E0F5301224427BFF7A16CA
:103D3F0079BC906100E0F5301224427BFF7A16794E
:103D4F00D3906414E0FEA3E0FFE48F338E32F5319D
:103D5F00F5301224427BFF7A1679F290618CE0FEE7
:103D6F00A3E0FFE48F338E32F531F5301224427B1E
:103D7F00FF7A17791290618AE0FEA3E0FFE48F3398
:103D8F008E32F531F5301224427BFF7A177932905B
:103D9F006629E0FEA3E0FFE48F338E32F531F53074
:103DAF001224427BFF7A177951A205E433F53012C2
:103DBF0024427BFF7A17796EA204E433F530122484
:103DCF00427BFF7A177997A20BE433F53012244226
:103DDF007BFF7A1779BEA212E433F5301224427BAF
:103DEF00FF7A1779E2A20AE433F5301224427BFFFF
:0E3DFF007A1779FE906678E0F53012244222A1
:1032F6007E187F23125011EF4E70037F0122E49057
:103306006F5EF07E187F26125011EF4E601512592F
:1033160032BF3106906F5E740AF0BF3206906F5E60
:103326007464F07E187F2C125011EF4E600812550F
:103336007990618FEFF07E187F32125011EF4E6058
:1033460008125579906102EFF07E187F38125011FD
:10335600EF4E6008125579906101EFF07E187F3EBE
:10336600125011EF4E600D125579EC4D4E4F24FF61
:1033760092018002C2017E187F44125011EF4E6006
:1033860023125579A804A905AA06AB077F007E8CEF
:103396007D0A7C001227F51228879068B9EEF0A303
:1033A600EFF0800A9068B974FDF0A374C0F07E183F
:1033B6007F4A125011EF4E600A125579906413EF4E
:1033C600F080069064137401F07E187F501250113D
:1033D600EF4E600A125579906100EFF08008906414
:1033E60013E0906100F07E187F56125011EF4E6088
:1033F6000D125579906414EEF0A3EFF080089064F6
:1034060014E4F0A304F07E187F5C125011EF4E60B6
:103416000D12557990618CEEF0A3EFF0800A906161
:103426008C7403F0A374E9F07E187F62125011EFDA
:103436004E600D12557990618AEEF0A3EFF0800A86
:1034460090618A740BF0A374B9F07E187F681250ED
:1034560011EF4E600D125579906629EEF0A3EFF04C
:10346600800A9066297407F0A374D1F07E187F6EE7
:10347600125011EF4E600D125579EC4D4E4F24FF50
:1034860092058002C2057E187F74125011EF4E60BD
:103496000D125579EC4D4E4F24FF920B8002C20B54
:1034A6007E187F7A125011EF4E600D125579EC4D51
:1034B6004E4F24FF92048002C2047E187F80125071
:1034C60011EF4E600D125579EC4D4E4F24FF9209C7
:1034D6008002D2097E187F86125011EF4E600D12BF
:1034E6005579EC4D4E4F24FF92128002D2127E186F
:1034F6007F8C125011EF4E600A125579906678EF64
:10350600F080069066787401F07E187F9212501152
:10351600EF4E600D125579EC4D4E4F24FF920A8006
:0535260002C20A7F0053
:01352B00227D
:10352C009069C0E064557004A3E064816064E4F5C4
:10353C006B741F256BF582E43466F583E4F0741626
:10354C00256BF582E43466F583E4F0740A256BF59B
:10355C0082E43463F583E4F0056BE56BB408D2E4E4
:10356C00F56B7479256BF582E43467F583E4F0052B
:10357C006BE56BB440ECE4F56B74C2256BF582E43F
:10358C003461F583E4F0056BE56BB480ECE4F56D28
:10359C00F56CE490718CF0C203C208906628F0C2FE
:1035AC0011C207C210C202C206F56B90618EF0F513
:1035BC0062906187F0F569F573C200C213C20D9079
:1035CC0068B974FFF0A374F4F07565FF9061017431
:1035DC0002F0A3F090618FF01232F6E4F5129071C4
:1035EC00887461F0A37490F090618FE0F512E5128D
:1035FC00C394014007E512D394084003E4F512E5A7
:10360C00126028907188E475F0011227A385F0826E
:10361C00F58374C4F01512907188E475F0011227CB
:10362C00A385F082F583E512F080D4906102E0F579
:10363C0012E512C394014007E512D394084003E449
:10364C00F512E5126028907188E475F0011227A339
:10365C0085F082F58374C8F01512907188E475F0CA
:10366C00011227A385F082F583E512F080D49061D6
:10367C0001E0F512E512C394014007E512D394085A
:10368C004003E4F512E5126028907188E475F001AE
:10369C001227A385F082F58374C2F01512907188FD
:1036AC00E475F0011227A385F082F583E512F08012
:1036BC00D4907188E475F0011227A385F082F5830C
:1036CC00E4F090718875F0011227A385F082F583E0
:1036DC00E4F0F512C291C290C2ADF5C9D2CDD2CCF4
:1036EC00C2C9C2CAF5CDF5CC9068B9E0F5CBA3E060
:1036FC00F5CA85CBCD85CACCD29FD29ED29CD2CADC
:10370C00C2ACC298C29975B81075B710D2AC12542D
:01371C005458
:01371D002289
:024C61008F2E94
:104C6300E4FF7C617D03FEEEC3952E50120DEDAA89
:104C73000470010C14F5828A83E02FFF0E80E80D87
:104C8300EDAA0470010C14F5828A83EFF00DEDAEEA
:104C93000470010C14F5828E837416F0052E052E14
:104CA3007E677FB97C617D03E52EB4040E8F828E0F
:104CB300837410F00FBF00010E80328F828E8374D5
:104CC30068F00FBF00010EE52E24FEFB8F828E835A
:104CD300F00FBF00010E8F828E83EBF00FBF000138
:104CE3000E8F828E837468F00FBF00010E8C838D4C
:104CF3008263A2018E838F8263A201AF2E1237F9E2
:0D4D0300E52EB4040304FF22E52E2404FF76
:014D10002280
:10570200200335124C6190618EEFF030210B7E67E1
:105712007FB9E0FDE4FB1248A5300D057F01125967
:105722009DE5626003F57022E490661EF0F56BD28F
:0957320003C2992099FDD29922CD
:022D49008F29D0
:102D4B00E54A30E714E54DB4100F201F077E187FBE
:102D5B00981246AAE4906187F0E54A24BE700302FC
:102D6B002FF124FA7003022EEA24046003023024AC
:102D7B00E54B30E703022E13E54D6066E54CC3943B
:102D8B00024003023024E54C7007E54D14F52A8010
:102D9B0006E54D241FF52AE52A75F004A42413F546
:102DAB0082746335F0F5837D4F7F041237E7E52A94
:102DBB0075F004A4240AF582746235F0F5837D5313
:102DCB007F041237E77402254CF582E43462F583F5
:102DDB007481F074C2252AF582E43461F5837401A1
:102DEB00F0227416254CF582E43466F583E04481B9
:102DFB00F0E54C25E025E0244CF582E43466F583C0
:102E0B007D4F7F041237E722E54E640860030230E2
:102E1B0024752901E54D5407FFE529A80708800211
:102E2B00C333D8FCF5297408256DF56DB56C0674A4
:102E3B0008256CF56CE54D547FFFE54CC43354E02D
:102E4B002FFE7400256DF582E43460F583EEF0E51A
:102E5B004DC39480503CEF131313541FFFE54C25C7
:102E6B00E025E025E025E0244CF582E43466F5838B
:102E7B00E5822FF582E43583F583E0FFE529F4FE47
:102E8B00EF5EF07401256DF582E43460F583E4F0B8
:102E9B00803AE54D547FFF131313541FFFE54C2568
:102EAB00E025E025E025E0244CF582E43466F5834B
:102EBB00E5822FF582E43583F583E04529F0740133
:102ECB00256DF582E43460F5837401F07402256D91
:102EDB00F582E43460F5837D4F7F061237E722E5F8
:102EEB004D54E06440702CE54D540F144440FF7476
:102EFB000A254CF582E43463F583EFF0E54C25E0CD
:102F0B0025E0242BF582E43466F5837D4F7F041294
:102F1B0037E722740A254CF582E43463F583E0F538
:102F2B000CE54D547FFF1313543FF50AE50C30E6C7
:102F3B0077540FB50A2D301216E50C54074490FE4A
:102F4B00740A254CF582E43463F583EEF08014E5C6
:102F5B000C54074410FE740A254CF582E43463F5D7
:102F6B0083EEF030122175F008E54CA4250AF582AA
:102F7B00E435F0F583E5822479F582E5833467F552
:102F8B0083E054FEF0804075F008E54CA4250AF56B
:102F9B0082E435F0F583E5822479F582E5833467A5
:102FAB00F583E04403F0801F75F008E54CA4250A77
:102FBB00F582E435F0F583E5822479F582E58334F7
:102FCB0067F583E04403F075F040E54CA42416F557
:102FDB0082E5F03464F58375F002EF1229037D4F1F
:102FEB00AF4E1237E722302D30E54DB40112201FC2
:102FFB00077E187FA41246AAE55004907077F02242
:10300B00E54DB4031490705FE0B401037405F02038
:09301B001F077E187FAF1246AAC0
:013024002289
:101F240020140302201B9080E8E0700F12545430F8
:101F340021077E187FBB1246AAC20C9080E8E06499
:101F44000E6003021FE4200A03021FCF9080F0F00A
:101F5400906185E0FF04F0EF30E025906C0BE0FF2A
:101F640060419080F0F0906C0CE09080F1F0906C07
:101F74000DE09080F2F0906C0EE09080F3F08023FE
:101F8400906C0FE0FF601C9080F0F0906C10E0907B
:101F940080F1F0906C11E09080F2F0906C12E0907F
:101FA40080F3F07529099080F4E529F0752964A37C
:101FB400E529F09080F0E060229080037404F03012
:101FC40021197E187FC41246AA80109080037408D9
:101FD400F03021077E187FD01246AAC20C756355D3
:101FE4009080E8E0B4060D200C0A3021077E187FAB
:101FF400DB1246AAE56A6002156AC214302D1890F5
:102004006186E004F0E0D39414400C201F077E188E
:102014007FF11246AAC22D906628E0704B90664B61
:10202400E004F0E0FFD394074007E56360037563C1
:1020340003EF540790664BF0E0FF240AF582E43482
:1020440063F583E0FE30E720740A2FF582E43463FD
:10205400F583EE547FF0740A2FF582E43463F5833C
:10206400E0540F04906628F020112A906188E0045F
:10207400F0E0543FF0E0FF2479F582E43467F5831F
:10208400E0FE30E010D21174792FF582E43467F564
:1020940083EE54FEF0200726906627E004F0E05417
:1020A4003FF0E0FF24C2F582E43461F583E0600E82
:1020B400D20774C22FF582E43461F583E4F020087A
:1020C4002A906189E004F0E05407F0E0FF2416F55B
:1020D40082E43466F583E0FE30E71074162FF5824F
:1020E400E43466F583EE547FF0D208300C63E56A7D
:1020F400705F7E707F82120EF08F29E52960529006
:10210400707EE561F0E560A3F0A3E55FF0E55EA312
:10211400F03005020529300B020529300402052997
:10212400E529240490707DF0E5292406FF124A8BEA
:1021340074022561F561E43560F560906312E00492
:10214400F0906678E0FF906312E0C39F4003756AE5
:10215400041249998F29E5297003022210302112B3
:102164007E187FFF1246AA7E707F7CE4FBAD2912A5
:1021740048A590707EE0B4071C740BF07F06124AE9
:102184008BE4F560F561F55EF55FD20CF56A90635A
:1021940012F075635590707EE0B443087483F07F49
:1021A40006124A8B90707EE0B4130A7423F07F0603
:1021B400124A8BC20C90707EE0FFB40107E4F56A0A
:1021C400906312F0EF20E04690707D7404F0A3E079
:1021D400752C00F52DA3E0FEE4EE422C7402252DAF
:1021E400F52DE4352CF52C90707E7401F0E4A3F009
:1021F400A3E52DF0E52CA3F07F06124A8B852C5E17
:10220400852D5F7E707F82122A568002C21E2006B0
:10221400030223DFE56F54802479F582E43466AF4A
:1022240082F52A8F2B3021157E197F041246AAE5E8
:102234006F547FFDE4FBAF2BAE2A1248A5200E0697
:10224400200F030223DD852B82852A83A3E0FF90E0
:102254006413E0FEEF6E60030223D9E52B2407F537
:1022640082E4352AF583E0FEE52B2406F582E43585
:102274002AF583E07C002400F52DEC3EF52C852B1B
:1022840082852A83E0544F24BF604624FE60641490
:10229400700302232C24FB700302234514700302F1
:1022A4002364147003022364240B60030223CF20ED
:1022B4001F077E197F071246AAE4906103F0906419
:1022C40013E0906104F07F021257027563550223F4
:1022D400D9201F077E197F1D1246AAE4906103F0DE
:1022E400906413E0906104F07F0212570275635505
:1022F4000223D9201F077E197F041246AAE49061A5
:1023040003F0906413E0906104F07F0212570220FE
:102314001F077E197F351246AAE52B2402FFE435F8
:102324002AFE122A560223D9201F077E197F04127F
:1023340046AAE52B2402FFE4352AFE122A5602237C
:10234400D9201F077E197F3D1246AA906103740BA2
:10235400F0906413E0906104F07F021257028075DC
:10236400201F077E197F551246AA906187E0C39407
:10237400055005E004F0805D7E617F05120EF08F4C
:1023840029E52960279061037408F0906413E090B4
:102394006104F03005020529300B020529300402DE
:1023A4000529E5292402FF1257028029906103744C
:1023B40009F0906413E0906104F07F021257022048
:1023C4001F137E197F5F1246AA800A201F077E19F9
:0B23D4007F6C1246AAC20FC20EC206A8
:0123DF0022DB
:102A56008E2E8F2F8F828E83E0249C7003022C96FD
:102A660024FD7003022BB1243A6003022D48201F77
:102A7600077E197F721246AA852E83852F8263A24E
:102A86000190666C63A2017F0B1237F9852F828550
:102A96002E83A3A3E0543FF50A7403252FF52FE4F4
:102AA600352EF52E300408052FE52F7002052E85EC
:102AB6002F82852E83E0FF906100E0FEEF6E6003BB
:102AC600022D48052FE52F7002052E300508052F2B
:102AD600E52F7002052E852F82852E83E075660010
:102AE600F567052FE52F7002052EF582852E83E00A
:102AF600FEE4EE4266052FE52F7002052E9066294C
:102B0600E0FEA3E0FFC3E5679FF567E5669EF56611
:102B1600D3E5679480E56694004003022D48300BA8
:102B260008052FE52F7002052E852F82852E83E05E
:102B3600F50CE50A64067066E50C30E742201F07CF
:102B46007E197F771246AA302D03022D48D22DE436
:102B560090705FF0906186F0E566C4F854F0C8683E
:102B6600E567C4540F48907060F0E567540F25E0A0
:102B7600FFE433E50C640154012F907065F02220C8
:102B86001F077E197F7F1246AA202D03022D48902B
:102B9600705FE064066003022D487402F022201F75
:102BA600077E197F8B1246AAC22D22201F077E1987
:102BB6007F941246AA906187740AF07406252FF551
:102BC6002FE4352EF52E300508052FE52F7002056A
:102BD6002E300B08052FE52F7002052E3004080550
:102BE6002FE52F7002052E052FE52FAE2E7002055C
:102BF6002E14F5828E83E0756600F567052FE52FA6
:102C0600AE2E7002052E14F5828E83E0FEE4EE42AF
:102C160066052FE52FAE2E7002052E14F5828E83E3
:102C2600E0F50C052FE52FAE2E7002052E14F58269
:102C36008E83E0F50B052FE52FAE2E7002052E14C0
:102C4600F5828E83E0F50A052FE52FAE2E7002057C
:102C56002E14F5828E83E0F50D052FE52FAE2E702E
:102C660002052E14F5828E83E0F508AE66AF677C0A
:102C7600037DE812274E8F09124375907061E511A6
:102C8600F0A3E510F0A3E50FF0A3E50EF0D22F2296
:102C9600201F077E197F9C1246AAE5636003022D5A
:102CA60048852F82852E83A3A3E064066003022D48
:102CB600487406252FF52FE4352EF52E3005080528
:102CC6002FE52F7002052E300B08052FE52F700219
:102CD600052E300408052FE52F7002052E852F825C
:102CE600852E83E06414705AE4F50C7416250CF5F1
:102CF60082E43466F583E030E00E7416250CF58226
:102D0600E43466F5837483F0740A250CF582E434A2
:102D160063F583E0FF30E40F740A250CF582E43492
:102D260063F583EF44A0F0050CE50CB408BD906193
:102D36008974FFF090664BF0E4906628F0C208753F
:032D460063012204
:105837008E318F32300404E4123809906100E0128F
:105847003809300504E4123809E532123809E53120
:0B585700123809300B04E4123809225B
:040EF0008E2E8F2F84
:100EF400E56364557036201F077E197FA41246AA45
:100F040063A201852E83852F8263A201E4F56374B5
:100F14004612380974011238097404123809E4FFBE
:100F2400FE12583774021238097F0722202D03025B
:100F34000FFD907077E0605190666C63A201852E7E
:100F440083852F8263A2017F0B1237F9907077E0BB
:100F5400B40117201F077E197FBE1246AA852F826F
:100F6400852E83A3A3740AF08015201F077E197FA2
:100F7400C71246AA852F82852E83A3A37447F0E463
:100F8400907077F0C22D7F072290705FE064057047
:100F940031201F077E197FD21246AA90666C63A285
:100FA40001852E83852F8263A2017F091237F9857B
:100FB4002F82852E83A3A37407F090705F14F07FB3
:100FC400072290705FE06403702F201F077E197F53
:100FD400DE1246AA90666C63A201852E83852F8259
:100FE40063A2017F091237F9852F82852E83A3A37B
:100FF4007407F090705FF0FF22E56D656C7003027A
:1010040010D5201F077E197FED1246AAE56C24082F
:10101400F5307408256CF56CD21374022530F58212
:10102400E43460F583E0F51174032530F582E4348B
:1010340060F583E0F51074042530F582E43460F53E
:1010440083E0F50F74052530F582E43460F583E020
:10105400F50E124240AF097E007C037DE812273C66
:101064008E668F6763A201852E83852F8263A2011A
:10107400741E123809740112380974031238097481
:10108400002530F582E43460F583E0FF906415E0D8
:101094002FFF906414E03400FE1258377401253099
:1010A400F582E43460F583E0123809E56712380903
:1010B400E566123809E50C123809E50B123809E522
:1010C4000A123809E50D123809E5081238097F0EAD
:1010D40022E56330E045201F077E197FF31246AAFC
:1010E40063A201852E83852F8263A2017464123862
:1010F400097401123809E563B4010A740712380946
:101104007563028008740A123809E4F563E4FFFE8B
:1011140012583774141238097F0722200803021169
:10112400D5201F077E1A7F011246AAC20863A201B6
:10113400852E83852F8263A201740112380974A05D
:10114400123809906189E02416F582E43466F58347
:10115400E030E1187414123809906189E02416F51E
:1011640082E43466F583E054FDF08005740212389D
:1011740009906189E075F020A4FF906415E02FFFC9
:10118400906414E035F0FE125837E4F5309061892C
:10119400E025E025E0244CF582E43466F583E5821D
:1011A4002530F582E43583F583E0F50AE4F50CE5B2
:1011B4000A5401123809E50AC313F50A050CE50CB3
:1011C400C3940840EA0530E530C3940440BF7F2649
:1011D40022906628E07003021368201F077E1A7F9E
:1011E400071246AA906628E025E025E0F50CE4F015
:1011F40063A201852E83852F8263A20190664BE052
:10120400FF240AF582E43463F583E0FE30E55B7481
:101214000A2FF582E43463F583EE54DFF074091287
:101224003809E50C248012380974141238099066C0
:101234004BE075F020A4FF90618DE02FFF90618C4E
:10124400E035F0FE12583790664BE075F040A42468
:1012540016F582E5F03464F583AF0C123812E50C10
:1012640075F003A4F5302406FF2230121374221201
:101274003809E50C248012380974031238098011E6
:101284007409123809E50C248012380974011238E3
:101294000990664BE075F020A4FF90618DE02FFF6C
:1012A40090618CE035F0FE12583790664BE075F093
:1012B40040A42416F582E5F03464F583AF0C1238AB
:1012C40012E50C75F003A4F5302012030213622515
:1012D4002FF52FE4352EF52E90664BE0FF25E02503
:1012E400E0242BF582E43466F583E0F511EF25E084
:1012F40025E0242CF582E43466F583E0F51090664D
:101304004BE0FF25E025E0242DF582E43466F583E7
:10131400E0F50FEF25E025E0242EF582E43466F5B0
:1013240083E0F50E124240AF097E007C037DE81293
:10133400273C8E668F67EF123809E566123809E597
:101344000C123809E50B123809E50A123809E50DC3
:10135400123809E508123809E530240DFF22E5307A
:101364002406FF2220070302147F201F077E1A7F12
:101374000E1246AAC20763A201852E83852F8263BB
:10138400A201742512380974011238097401123843
:1013940009906627E0FF90618BE02FFF90618AE05F
:1013A4003400FE125837906627E025E025E0F5303A
:1013B400FF053074132FF582E43463F583E01238AB
:1013C40009AF30053074132FF582E43463F583E0FC
:1013D400123809AF30053074132FF582E43463F505
:1013E40083E0123809AF30053074132FF582E434EA
:1013F40063F583E0123809E412380974FC2530F5EA
:1014040030FF0530740A2FF582E43462F583E0F589
:1014140011AF300530740A2FF582E43462F583E0AD
:10142400F510AF300530740A2FF582E43462F58389
:10143400E0F50FAF300530740A2FF582E43462F51D
:1014440083E0F50E124240AF097E007C037DE81272
:10145400273C8E668F67EF123809E566123809E576
:101464000C123809E50B123809E50A123809E50DA2
:10147400123809E5081238097F122230115A201F48
:10148400077E1A7F141246AAC21163A201852E8315
:10149400852F8263A20174091238097484123809F1
:1014A4007402123809906188E075F004A4FF906119
:1014B4008DE02FFF90618CE035F0FE12583790617B
:1014C40088E075F008A42416F582E5F03464F58309
:0A14D4007F041238127F12227F00FD
:0114DE0022EB
:0100220022BB
:104F91000208A4E493A3F8E493A34003F68001F28A
:104FA10008DFF48029E493A3F85407240CC8C33321
:104FB100C4540F4420C8834004F456800146F6DFF0
:104FC100E4800B01020408102040809059A6E47E81
:104FD100019360BCA3FF543F30E509541FFEE493E5
:104FE100A360010ECF54C025E060A840B8E493A3AC
:104FF100FAE493A3F8E493A3C8C582C8CAC583CAD7
:10500100F0A3C8C582C8CAC583CADFE9DEE780BE8E
:0159AC0000FA
:10273C00EF8DF0A4A8F0CF8CF0A428CE8DF0A42EB1
:02274C00FE226B
:10274E00BC000BBE0029EF8DF084FFADF022E4CC6F
:10275E00F875F008EF2FFFEE33FEEC33FCEE9DEC38
:10276E00984005FCEE9DFE0FD5F0E9E4CEFD22ED7E
:10277E00F8F5F0EE8420D21CFEADF075F008EF2FC8
:10278E00FFED33FD4007985006D5F0F222C398FDB9
:05279E000FD5F0EA2256
:1027A300A3F8E0C5F025F0F0E582158270021583E9
:0627B300E0C838F0E82246
:1027B90075F008758200EF2FFFEE33FECD33CDCCD7
:1027C90033CCC58233C5829BED9AEC99E58298405A
:1027D9000CF582EE9BFEED9AFDEC99FC0FD5F0D637
:1027E900E4CEFBE4CDFAE4CCF9A88222B800C1B961
:1027F9000059BA002DEC8BF084CFCECDFCE5F0CB9F
:10280900F97818EF2FFFEE33FEED33FDEC33FCEBD7
:1028190033FB10D703994004EB99FB0FD8E5E4F992
:10282900FA227818EF2FFFEE33FEED33FDEC33FC7F
:10283900C933C910D7059BE99A4007EC9BFCE99A73
:10284900F90FD8E0E4C9FAE4CCFB2275F010EF2FB8
:10285900FFEE33FEED33FDCC33CCC833C810D707B8
:102869009BEC9AE899400AED9BFDEC9AFCE899F8F3
:0E2879000FD5F0DAE4CDFBE4CCFAE4C8F92286
:0E288700C3E49FFFE49EFEE49DFDE49CFC2262
:10289500EB9FF5F0EA9E42F0E99D42F0E89C45F099
:0128A5002210
:1028A600E493FC740193FD740293FE740393FF2278
:1028B600E493F8740193F9740293FA740393FB2278
:0C28C600ECF0A3EDF0A3EEF0A3EFF02285
:1028D200A8828583F0D083D0821228E91228E912D7
:1028E20028E91228E9E473E493A3C583C5F0C583FC
:1028F200C8C582C8F0A3C583C5F0C583C8C582C850
:0129020022B2
:0C290300A42582F582E5F03583F58322DF
:1023E000E53C2430F8E6053C22782D302B0278308D
:1023F000E475F0011229B602290F2024EB7F2ED2BA
:10240000248018EF540F2490D43440D4FF30280B8C
:10241000EF24BFB41A0050032461FFE53D600215AC
:102420003D0540E5407002053F302B0D782DE475E9
:10243000F0011229B6EF02295502562F7403D22B50
:102440008003E4C22BF53C8B2D8A2E892FE4F53DC9
:10245000F53FF540E53D60077F2012241B80F575B0
:102460003EFFC225C224C226C227C229C22AC22CCC
:102470001223E9FF700D302B057F0012242CAF4092
:10248000AE3F22B4255FC2D5C2281223E9FF24D073
:10249000B40A00501A75F00A783D30D50508B6FF29
:1024A0000106C6A426F620D5047002D22780D924BE
:1024B000CFB41A00EF5004C2E5D22802262CD22550
:1024C00080C6D22480C0D22680BCD2D580BAD22980
:1024D00080B47F2012241B2026077401B53D0040E4
:1024E000F11223E0FF12241B022454D22CD22A80A2
:1024F000951223E0FB1223E0FA1223E0F94A4B7015
:102500000679FD7A267BFF20262EE53D602A7E0097
:102510008E8275830012292860060EEE653E70F0EB
:10252000C2D5EBC0E0EAC0E0E9C0E0EE122673D00D
:10253000E0F9D0E0FAD0E0FB12290FFF60AAEBC06F
:10254000E0EAC0E0E9C0E012241BD0E02401F9D0A9
:10255000E03400FAD0E0FBE53E0460DCD53ED980F3
:10256000877BFF7A26796FD226809C79108002794A
:1025700008C22AC22C8008D2D5790A8004790AC2FE
:10258000D5E53E047002F53EE4FAFDFEFF1223E0BD
:10259000FC7B082025131223E0FD7B1030240A1257
:1025A00023E0FE1223E0FF7B20EC3382D592D5504E
:1025B00013C3E43024069FFFE49EFEE42025039D20
:1025C000FDE49CFCE4CBF8C225EC700CCFCECDCC66
:1025D000E824F8F870F38017C3EF33FFEE33FEED15
:1025E00033FDEC33FCEB33FB994002FB0FD8E9EBF6
:1025F000302505F8D0E0C448B225C0E00AEC4D4EC5
:102600004F78207B0070C2EAB53E0040BCC0E012AB
:102610002675D0F0D0E0202504C4C0E0C4B225C0A7
:10262000F0122404D0F0D5F0EB022454122A152421
:10263000F153256B5824C24C24BE42256F4F257799
:0F2640004425774924D743257D552561462561DB
:10264F0045256147271D5024C62D24CA2E24ED2B66
:10265F0024CE2324EB2027062A248648000024E5D5
:10266F003F3F3F00790AA2D5202714302909B9101E
:10267F00020404B9080104A2D5202A025001042043
:10268F0026689226B53D005034C0E07F20302719D0
:10269F007F30A226722A7229500F1226CCC226C270
:1026AF002AC229C22C7F30800F302903E9C0E012E3
:1026BF00241B302903D0E0F9D0E0B53DCC302917E9
:1026CF007F30B9100C12241B7F583028077F788079
:1026DF0003B9080312241B3026057F2D02241B7F0C
:1026EF0020202CF87F2B202AF322922680CF286ED1
:1026FF00756C6C2900D2251223E03025F8C225789D
:10270F003D30D50108F60224862D50434958122337
:10271F00E02403B405004001E49027189312240C21
:0D272F00743A12240CD227753D0402256B6C
:103ADB008B2D8A2E892FE4F539F538F537F536F528
:103AEB0034F535E531453245306012EBC0E0EAC0C4
:103AFB00E0E9C0E0AB30AA31A9321229C6AB2D05E3
:103B0B002FE52FAA2E7002052E14F912290FF53A64
:103B1B00C394094007E53AD3940D40E1E53A64209C
:103B2B0060DBE53AB42D054335038016E53AB42B3B
:103B3B0005433501800C74FF252FF52F74FF352EAF
:103B4B00F52EE53360046410703FAB2DAA2EA92F20
:103B5B0012290F64306009E533702E75330A802902
:103B6B00900001122928FF64786004EFB4581343C6
:103B7B0035017533107402252FF52FE4352EF52EF4
:103B8B008007E5337003753308AB2D052FE52FAA9E
:103B9B002E7002052E14F912290FF53AC3946140C9
:103BAB000AE53AD3947A5003533ADF74D0253AF5A9
:103BBB003AC3940A400CE53A9411406D74F9253AD6
:103BCB00F53AE53AD39533506043350185393E8557
:103BDB00383D85373C85363BAF337E00E4FCFDAB8F
:103BEB0039AA38A937A836122967C8ECC8C9EDC954
:103BFB00CAEECACBEFCBE4FCFDFEEB253AF539EE72
:103C0B003AF538ED39F537EC38F536AF39AE38AD26
:103C1B0037FCAB3EAA3DA93CA83BD31228955003D9
:103C2B00023B94433504023B94E53520E003E480EA
:103C3B002DE53145324530601EAB2DE52F24FFF9C4
:103C4B00E52E34FFFAEBC0E0EAC0E0E9C0E0AB30B0
:103C5B00AA31A9321229C6E53530E20774FFFFFEFF
:103C6B00FDFC22E535AF39AE38AD37AC3630E1036C
:043C7B000228872272
:10290F00BB010689828A83E0225002E722BBFE02C6
:09291F00E32289828A83E49322F9
:10292800BB010CE58229F582E5833AF583E0225064
:1029380006E92582F8E622BBFE06E92582F8E222AE
:0D294800E58229F582E5833AF583E49322C8
:10295500BB010689828A83F0225002F722BBFE0161
:02296500F3225B
:10296700E88FF0A4CC8BF0A42CFCE98EF0A42CFC0F
:102977008AF0EDA42CFCEA8EF0A4CDA8F08BF0A48D
:102987002DCC3825F0FDE98FF0A42CCD35F0FCEBEC
:102997008EF0A4FEA9F0EB8FF0A4CFC5F02ECD39B1
:0F29A700FEE43CFCEAA42DCE35F0FDE43CFC221E
:1029B600FAE6FB0808E6F925F0F618E6CA3AF62222
:1029C600BB011A89828A83D0F0D0E0F8D0E0F9D032
:1029D600E0FAD0E0FBE8C0E0C0F0022A445016E975
:1029E600F8D083D082D0E0F9D0E0FAD0E0FBC08204
:1029F600C083022A3BBBFE16E9F8D083D082D0E022
:0F2A0600F9D0E0FAD0E0FBC082C083022A4D2253
:102A1500D083D082F8E4937012740193700DA3A350
:102A250093F8740193F5828883E473740293686064
:062A3500EFA3A3A380DF64
:092A3B00EBF608EAF608E9F622C0
:092A4400EBF0A3EAF0A3E9F02293
:092A4D00EBF208EAF208E9F222BA
:00000001FF
